S02B000062696E2F6F70656E626C745F64656D6F70726F675F6E75636C656F5F73746D33326631303372622EC3
S31508000000F4060020F90F0008DD0F0008DD0F0008D0
S31508000010DD0F0008DD0F0008DD0F0008DD0F000802
S31508000020DD0F0008DD0F0008DD0F0008DD0F0008F2
S31508000030DD0F0008DD0F0008DD0F0008DD0F0008E2
S31508000040DD0F0008DD0F0008DD0F0008DD0F0008D2
S31508000050DD0F0008DD0F0008DD0F0008DD0F0008C2
S31508000060DD0F0008DD0F0008DD0F0008DD0F0008B2
S31508000070DD0F0008DD0F0008DD0F0008DD0F0008A2
S31508000080DD0F0008DD0F0008DD0F0008DD0F000892
S31508000090DD0F0008DD0F0008DD0F0008DD0F000882
S315080000A0DD0F0008DD0F0008DD0F0008DD0F000872
S315080000B0DD0F0008DD0F0008DD0F0008DD0F000862
S315080000C0DD0F0008DD0F0008DD0F0008DD0F000852
S315080000D0DD0F0008DD0F0008DD0F0008DD0F000842
S315080000E0DD0F0008DD0F0008DD0F0008DD0F000832
S315080000F0DD0F0008DD0F0008DD0F0008DD0F000822
S31508000100DD0F0008DD0F0008DD0F0008DD0F000811
S31508000110DD0F0008DD0F0008DD0F0008DD0F000801
S31508000120DD0F0008DD0F0008DD0F0008DD0F0008F1
S31508000130DD0F0008DD0F0008DD0F0008DD0F0008E1
S31508000140DD0F0008DD0F0008DD0F0008DD0F0008D1
S3150800015000B583B00023009301934FF48053C4F293
S3150800016002031A6842F001021A6059680022CFF6A3
S31508000170FF020A405A601A6822F0847222F480321A
S315080001801A601A6822F480221A605A6822F4FE025B
S315080001905A604FF41F029A601A6842F480321A6055
S315080001A04FF48053C4F2020340F2DC52196801F49A
S315080001B000310191009901310091019911B9009915
S315080001C09142F3D14FF48053C4F202031B6813F42F
S315080001D0003F06D141F25400C0F600006E2100F03F
S315080001E0FDFA4FF40053C4F202031A6842F01002F3
S315080001F01A601A6822F003021A601A6842F00202AC
S315080002001A604FF48053C4F202035A685A605A6857
S3150800021042F400525A605A6842F480625A605A6838
S3150800022022F47C125A605A6842F4E8125A601A6834
S3150800023042F080721A604FF48053C4F202031A68BF
S3150800024012F0007FFBD04FF48053C4F202035A68C1
S3150800025022F003025A605A6842F002025A604FF4CA
S315080002608053C4F202035A6802F00C02082AFAD133
S315080002704FF48053C4F20203DA6942F40032DA61B9
S315080002809A6942F005029A614FF40063C4F20103C9
S315080002901A6822F470621A601A6842F430621A60A8
S315080002A01A6822F470421A601A6842F480421A6088
S315080002B000F004F800F010F8FCE700BF08B500F0FD
S315080002C091FA00F087FA00F0C7FB00F0A7FB00F0F0
S315080002D00DF800F06DFA08BD08B500F07DFA00F0DB
S315080002E0D7FB00F00FF800F043FA08BD08B500F098
S315080002F063F800F0CDFA40F20003C2F200030022D0
S315080003001A7008BD08B540F20400C2F2000000F0F9
S3150800031009FB01280BD140F20003C2F200030022B8
S315080003201A7040F20400C2F2000000F065F808BD39
S31508000330704700BF08B540F20003C2F200031B78FD
S3150800034013B9C9B200F0BAFA00F04EF808BD00BFFA
S3150800035040F20003C2F200031878022806D00328E8
S3150800036006D001280CBF082040207047002070479F
S315080003700020704740F20003C2F2000318780228F2
S3150800038006D0032806D001280CBF08204020704755
S31508000390002070470020704708B500F01BF808BD1C
S315080003A040F24403C2F20003FE22DA7018710222F8
S315080003B0A3F84420704700BF40F24403C2F200038A
S315080003C000221A709A6483F84320A3F844209A708E
S315080003D05A70704740F24403C2F20003187800309E
S315080003E018BF0120704700BF40F24403C2F2000361
S315080003F0002283F84320704738B504460178FF2960
S315080004001CD140F24404C2F20004002363700125A3
S315080004102570FF22E270102222716371FFF798FFA0
S31508000420A071FFF7A7FFE071FFF7A4FF000A20728B
S315080004306572A5720823A4F8443079E140F24403B2
S31508000440C2F200031B78012B40F09081C939352987
S3150800045000F26B81DFE811F0DB00690169016501D3
S31508000460690169015901FC0042012F01690169010D
S31508000470690169016901690169016901690169011E
S31508000480690169016901690169016901690169010E
S3150800049069016901690169016901690169016901FE
S315080004A06901690169016901690169017F005400EF
S315080004B036007300690169016901A1006901B90083
S315080004C0BD00CE004578FFF743FF0138854203DDBE
S315080004D02220FFF765FF2BE140F24405C2F2000532
S315080004E0281DA96C627800F09BF9FF23EB706278EF
S315080004F0AB6C1344AB6463780133A5F8443017E159
S315080005004578FFF725FF0138854203DD2220FFF7EE
S3150800051047FF0DE1616840F24405C2F20005A9648F
S31508000520281D627800F07CF9FF23EB706278AB6CCB
S315080005301344AB6463780133A5F84430F8E040F21D
S315080005404403C2F20003FF22DA7042689A64012269
S31508000550A3F84420ECE040F24403C2F20003FF2271
S31508000560DA709B6C406840B11844002213F8011BEE
S315080005700A44D2B28342F9D100E0002240F2440391
S31508000580C2F20003C3F8072001221A7100225A7129
S315080005909A710822A3F84420CAE040F24403C2F242
S315080005A00003FF22DA7041F25C02C0F600029A6488
S315080005B000221A715A719A710721D9711A725A72E0
S315080005C09A720822A3F84420B2E00020FFF7E8FE5A
S315080005D0AEE040F24403C2F20003FF22DA700022C2
S315080005E01A71597859719A71DA711A720622A3F832
S315080005F044209DE040F24403C2F2000300221A7030
S315080006005A70FF22DA700122A3F8442090E040F2E3
S315080006104403C2F200039D6CFFF79AFE411E28466A
S31508000620621C00F0FFF918B93120FFF7B9FE7FE028
S3150800063040F24404C2F20004FF23E370A56CFFF7FE
S3150800064087FE013D2844A0640123A4F844306FE0E6
S315080006504578FFF77DFE0238854203DD2220FFF745
S315080006609FFE65E040F24403C2F20003FF22DA70FF
S315080006700122A3F84420617839B900F0E3F900288B
S3150800068056D13120FFF78CFE52E040F24403C2F205
S315080006900003986CA21C00F0C5F918B93120FFF7C1
S315080006A07FFE45E040F24403C2F2000361789A6C8B
S315080006B00A449A643CE040F24404C2F20004FF2370
S315080006C0E370002525716571FFF742FEA071E5719B
S315080006D0257265720723A4F8443029E040F24403E2
S315080006E0C2F20003986C616800F0A0F918B93120CD
S315080006F0FFF756FE1CE040F24403C2F20003FF2255
S31508000700DA700122A3F8442012E000F06FF840F2F4
S315080007104403C2F20003FF22DA700122A3F8442040
S3150800072006E03120FFF73CFE02E02020FFF738FE06
S3150800073040F24403C2F2000393F84330012B02D17E
S315080007401020FFF72DFE40F24403C2F20003B3F86F
S3150800075044100BB2002B09DD40F24400C2F200003F
S31508000760012380F843300330FFF7E4FD38BD00BFAE
S3150800077008B5FFF711FE012819D040F29003C2F21E
S3150800078000031B78012B12D100F094F940F2940370
S31508000790C2F200031B6803F5FA73984207D340F2C6
S315080007A09003C2F2000300221A7000F01FF808BD79
S315080007B008B540F29003C2F2000301221A7000F055
S315080007C079F940F29403C2F200031860FFF7D0FFEC
S315080007D008BD00BF704700BF704700BF08B5FFF7E8
S315080007E0FBFFFCE708B500F003FC08BD10B500F0F8
S315080007F021F9A0B1FFF79CFD00F042F900F01EF9BF
S3150800080020F0604020F07F004EF60853CEF2000339
S31508000810186000F013F9446800F0ECFBA04710BD1F
S3150800082070B5561EB6B24AB14C1E0E44451A14F897
S31508000830013F2B55FFF7D0FFB442F8D170BD00BF7A
S3150800084010B54FF48843C4F200031B8803F08003F5
S315080008509BB2B3B14FF48843C4F2000398801B8857
S3150800086003F080039BB273B94FF48844C4F20004C2
S31508000870FFF7B2FF238803F080039BB2002BF7D063
S3150800088003E0002010BD012010BD012010BD00BFEF
S315080008904FF48843C4F2000300221A819A811A820F
S315080008A09A821A8340F271221A819A8992B242F484
S315080008B0005242F00C029A81704700BF2DE9F041C0
S315080008C006460C46402906D941F26400C0F60000E7
S315080008D08D21FFF783FF2046FFF7B2FF012806D0D8
S315080008E041F26400C0F600009121FFF777FF254624
S315080008F0ACB1002441F26407C0F600074FF09A082D
S31508000900FFF76AFF305DFFF79BFF012803D03846E3
S315080009104146FFF763FF0134A3B2AB42F0D3BDE80B
S31508000920F08100BF10B540F2E403C2F200031B7861
S315080009305BBB4FF48843C4F200031B8803F0200313
S315080009409BB2002B56D04FF48843C4F200039A8812
S3150800095092B240F2A003C2F200031A7012F0FF0F1F
S315080009604AD000F0A7F840F29803C2F200031860D4
S3150800097040F29C03C2F200030020187040F2E40320
S31508000980C2F2000301221A7010BD40F29C03C2F2A3
S3150800099000031A784FF48843C4F200031B8803F057
S315080009A020039BB263B34FF48843C4F200039C88C8
S315080009B040F2A003C2F2000399184C700132D2B279
S315080009C040F29C01C2F200010A701B78934215D1CD
S315080009D01149FFF725FF40F2E403C2F200030022A3
S315080009E01A70012010BD40F2E403C2F20003002091
S315080009F0187010BD002010BD002010BD002010BDCD
S31508000A0000F058F840F29803C2F200031B686433FA
S31508000A109842E8D8002010BDA100002008B500F0D3
S31508000A205BF908BD08B500F065F908BD08B500F022
S31508000A3089F908BD08B500F071FA08BD08B500F0D7
S31508000A40C7FA08BD08B500F03DFA10B100F09AFAE9
S31508000A5008BD002008BD00BF4EF21003CEF2000309
S31508000A6000221A6041F63F11C0F2010159609A60EE
S31508000A700521196040F2E803C2F200031A607047C4
S31508000A804EF21003CEF2000300221A60704700BF30
S31508000A904EF21003CEF200031B6813F4803F1FBF0B
S31508000AA040F2E803C2F200031A68013218BF1A605E
S31508000AB0704700BF08B5FFF7EBFF40F2E803C2F244
S31508000AC00003186808BD00BF4FF40053C4F20203C0
S31508000AD01A6942F080021A61704700BFF8B50746E6
S31508000AE00024254641F28C06C0F60006FFF774FE80
S31508000AF0A359BB420ED8311949680B449F4209D203
S31508000B0041F28C03C0F6000305EB450203EB8203B2
S31508000B10187AF8BD01350C349C2CE7D1FF20F8BDB6
S31508000B202DE9F84380460068FFF7D8FFFF285CD018
S31508000B304FF40053C4F2020340F22312C4F2675280
S31508000B405A6048F6AB12CCF6EF525A603422DA6095
S31508000B50DB6813F0010F04D0FFF7B6FF0020BDE8ED
S31508000B60F8834FF40053C4F202031A6942F00102F3
S31508000B701A61002508F104094FF40054C4F202046E
S31508000B80D8F80030EF1859F80560B2B2EA52E368AF
S31508000B9013F0010F05D0FFF71FFEE36813F0010FEE
S31508000BA0F9D1330C7B80E36813F0010F05D0FFF70A
S31508000BB013FEE36813F0010FF9D13B68B34204D181
S31508000BC00435B5F5007FDBD101E0002400E00124FF
S31508000BD04FF40053C4F202031A6922F001021A61A3
S31508000BE0FFF772FF2046BDE8F8830020BDE8F883CA
S31508000BF038B504460D4640F2EC03C2F200039842AB
S31508000C0009D04FF4C043C0F6000399420BD0FFF752
S31508000C1087FF20B917E040F2F024C2F20004C5F3BA
S31508000C20080393B903E040F2EC04C2F20004236817
S31508000C309D420CD0204640F8045B29464FF40072CA
S31508000C40FFF7EEFD03E0002038BD002038BD204642
S31508000C5038BD00BF2DE9F04106460C4617461D462D
S31508000C604FEA51284FEA48280368B3F1FF3F06D1F7
S31508000C7040F8048B41464FF40072FFF7D1FD336804
S31508000C80434505D030464146FFF7B2FF0646D0B188
S31508000C903368E41A3444043408F50078FFF79CFDF9
S31508000CA0331DE31AB3F5007F06D330464146FFF7F6
S31508000CB09FFF064650B1041D17F8013B04F8013B97
S31508000CC0013DEBD105E00020BDE8F0810020BDE83C
S31508000CD0F0810120BDE8F08140F2F023C2F2000362
S31508000CE04FF0FF321A6040F2EC03C2F200031A60BA
S31508000CF0704700BF70B504460D461646FFF7EEFE70
S31508000D00FF281BD0681E2044FFF7E8FEFF2817D0EF
S31508000D10620A4FF4C043C0F60003B3EB422F07BF85
S31508000D2040F2EC00C2F2000040F2F020C2F20000ED
S31508000D30214632462B46FFF78DFF70BD002070BD59
S31508000D40002070BD2DE9F84304460E46FFF7C6FE9F
S31508000D500546701E2044FFF7C1FE0446FF2D18BF46
S31508000D60FF2800F0AB80854200F29F80022D40F2FA
S31508000D709F800F2800F29F804FF40053C4F20203AD
S31508000D8040F22312C4F267525A6048F6AB12CCF608
S31508000D90EF525A603422DA60DB6813F0010F04D090
S31508000DA0FFF792FE0020BDE8F8834FF40053C4F223
S31508000DB002031A6942F002021A6141F28C09C0F66E
S31508000DC000094F460026FFF707FD3B7AAB4208D1DC
S31508000DD041F28C03C0F6000306EB460253F8227074
S31508000DE005E001360C370D2EEDD14FF0FF37C8461A
S31508000DF00025FFF7F1FC98F80830A34208D141F224
S31508000E008C03C0F6000305EB450253F8228006E082
S31508000E10013508F10C080D2DEBD14FF0FF384E4681
S31508000E200025FFF7D9FC337AA34209D141F28C0396
S31508000E30C0F6000305EB450203EB82035B6804E09A
S31508000E4001350C360D2DECD10023C7EB08084344B9
S31508000E50C3F38F23E3B1013B9EB20136B6020025E8
S31508000E604FF40054C4F20204EB196361236943F09A
S31508000E7040032361E36813F0010F05D0FFF7ACFCCC
S31508000E80E36813F0010FF9D105F58065B542EBD19A
S31508000E904FF40053C4F202031A6922F002021A61DF
S31508000EA0FFF712FE0120BDE8F8830020BDE8F883AD
S31508000EB00020BDE8F8830020BDE8F8830020BDE8DF
S31508000EC0F88300BF00B583B040F2EC03C2F200031A
S31508000ED01B68B3F1FF3F08BF01201CD040F2EC03AA
S31508000EE0C2F2000399685A681144DA6811441A690B
S31508000EF011445A6911449A690A44D96953185B42DC
S31508000F0002AA42F8043D46F25010C0F60000042139
S31508000F10FFF7F0FEFFE703B05DF804FB46F20402B4
S31508000F20C0F600024FF4C043C0F6000310681B6801
S31508000F30184446F20803C0F600031B68184446F234
S31508000F400C03C0F600031B68184446F21003C0F6EB
S31508000F5000031B68184446F21403C0F600031B6816
S31508000F60184446F21803C0F600031B68184446F2F4
S31508000F705013C0F600031B681844D0F1010038BFAF
S31508000F800020704708B540F2EC03C2F200031B6864
S31508000F90B3F1FF3F06D040F2EC00C2F20000FFF7C3
S31508000FA0BFFD88B140F2F023C2F200031B68B3F11B
S31508000FB0FF3F0BD040F2F020C2F20000FFF7B0FD71
S31508000FC0003018BF012008BD002008BD012008BD5B
S31508000FD04FF4C040C0F60000704700BF08B541F2A4
S31508000FE02810C0F600003121FFF7F8FB08BD00BF46
S31508000FF072B6704762B6704710B540F20002C2F288
S31508001000000240F20103C2F200039A4210D2131DF5
S315080010100D4CE41A24F0030404340023104641F26C
S315080010205811C0F600015A581A500433A342FAD18F
S31508001030064807494FF000028842B8BF40F8042B1B
S31508001040FADBFFF785F810BD040000200400002035
S31508001050F40400206D61696E2E6300004F70656EA2
S31508001060424C54002E2E2F2E2E2F2E2E2F536F75B8
S315080010707263652F41524D434D335F53544D33329E
S3150800108046312F756172742E6300000000600008F7
S315080010900020000003000000008000080020000077
S315080010A00400000000A00008002000000500000061
S315080010B000C00008002000000600000000E000084C
S315080010C000200000070000000000010800200000C2
S315080010D008000000002001080020000009000000A8
S315080010E000400108002000000A0000000060010816
S315080010F0002000000B00000000800108002000000E
S315080011000C00000000A00108002000000D000000EF
S3150800111000C00108002000000E00000000E00108E1
S31508001120002000000F0000002E2E2F2E2E2F2E2E10
S315080011302F536F757263652F41524D434D335F537D
S31508001140544D333246312F4743432F766563746FC8
S30D0800115072732E630000000013
S306080011580484
S70508000000F2
